:10000000C00AA4041C02160F43071B0A7C00E80761
:10001000140A09020A0143070F0A6700180AE900D7
:1000200089024306EA00180AAC0C2900040C2A00D5
:10003000070226002F0AA404BC021C028D014306FD
:100040004604A4041C028E014307280A0604260461
:10005000A4041C028F0143072F0A8604A604E106AC
:100060002F0AE20C2100000801096607390A01097C
:10007000350A4F0C2B000109EB004306430A010926
:1000800066073C0AAD0A0109DF0C2C00010966066F
:10009000500A01096606500A0109EC02470AAD0A36
:1000A0000109040C2B006607580A0109AB02530A28
:1000B00001090A0C8B000307AD0A01096606630AF1
:1000C0000109AB025E0A01093A0C8B000306AD0A76
:1000D0000109A404160224000B0220000109060CE9
:1000E0002B006607760A0109AB02710A01090C0CA4
:1000F0008B000307AD0A01096606810A0109AB02FC
:100100007C0A01093A0C8B000306AD0A0109A4041C
:10011000170224000B0220000109060C2B006607C1
:10012000940A0109AB028F0A01090C0C8B0003072A
:10013000AD0A010966069F0A0109AB029A0A010984
:100140003A0C8B000306AD0A0109A404180224002E
:100150000B0220000109E8040008E805340A6F00DA
:100160006F00C30C8F000307BB0A4307BF0A500C84
:100170008F000306BF0AAF024306AF02B10A0008B0
:1001800025006600080C0600080C0200E20C2100A5
:10019000AC0C2900040C2A006B006D006E006F008F
:1001A000390CA40433002A0C34002A0C35007C00DE
:1001B00068006700110C3600120C3700100C380074
:1001C000C804010934090109080428040109A40428
:1001D0001402F10101090304A40431030109A40478
:1001E000110234000109290CA40491000306FE0A3F
:1001F000010908052B0CA404B100710201092C0CA3
:10020000A40491000307090B010928052A0CA40482
:10021000B10001090304A40451032E000109C80719
:10022000150B4F0CA404B00070020109A4041302C2
:10023000F00101090304A40430030109A40410021D
:10024000330001091C0CA404900003062A0B0109C9
:100250004804300B010948051A0CA40490002D0035
:1002600001098804A8040109A4041502F201010986
:100270000304A40432030109A40412023500290C6A
:1002800092000306490B010988052B0CA404B20057
:10029000720201092C0CA40492000307540B0109FB
:1002A000A8052A0CA404B20001090304A404520303
:0A02B0002F00010908022700E10AEF
:021FFE00EA0FE8
:00000001FF
